:020000040000FA
:0600000063EF10F0120096
:06002A00010008210000A6
:08003000CA00000002000000FC
:08003800000100910093009506
:1000400000970D0E016F306BC00E036F330E046FFF
:10005000F10E056F8AEF03F0000102911CEF00F032
:1000600021DA46E822DA076EF450086E0A0ED890BC
:1000700008BE03D0075C000E085815E3083404E2FC
:1000800007500D08000E08540EE3CFD9030E035C91
:100090000AE1C00E04140001036F05EB04F006EB47
:1000A00005F0000E01D0010E47E9E7CFD9FF12009D
:1000B000F9D9000EEDD1F6D944E8F7D9056EF45020
:1000C000066E060ED89006BE03D0055C000E0658DC
:1000D00013E3063404E205500708000E06540CE34F
:1000E000A4D9030409E104EB01F00001015102E18C
:1000F0004C0E016F000E01D0010E45E9E7CFD9FF8C
:100100001200D0D9C5D18CD984E941E8046A0250E3
:10011000150A66E0060A61E0010A5BE0030A55E0A1
:10012000010A50E01E0A4BE0020A47E0070A42E0DB
:10013000010A3DE01E0A39E01D0A50E0010A32E0E2
:100140000F0A2DE0080A26E0090A21E00B0A1CE04C
:10015000080A17E0010A12E0070A0DE0010A09E0A7
:10016000030A03E0010A40E03DD085EC03F0090EEC
:100170003AD062DF39D00001009336D0000100830D
:1001800033D00001009130D0000100812DD0010E4C
:10019000E66E01D0E66A28EC03F041E924D00001C4
:1001A000009522D0000100851FD00B0E1CD000014D
:1001B00000971AD00001008717D0010E14D02BD958
:1001C0004FDF05D028D974DF02D025D974DF42E98A
:1001D0000AD021D996DF42E907D03EDF0A0E03D0CC
:1001E0000D0E01D0010E046E045042E9E7CFD9FF95
:1001F000120016D982E900500D0A42E0040A48E0D4
:10020000050A3AE0040A34E00F0A2EE0010A28E069
:10021000030A22E0010A1CE00F0A18E0010A12E0BA
:10022000080A0CE0020A06E0010A2CE1EA0EE66E7A
:100230001C0E2BD0EC0EE66E1C0E27D0C60EE66E02
:100240001C0E23D0EF0EE66E1C0E1FD0B3D820D0AC
:10025000060EE66E1D0E19D0110EE66E1D0E15D09F
:100260001D0EE66E1D0E11D0250EE66E1D0E0DD074
:100270002B0EE66E1D0E09D0340EE66E1D0E05D057
:100280008AD806D03D0EE66E1D0EE66E69D842E9AC
:10029000000EE66E1F0EE66E73EC0AF042E9F8D02F
:1002A00001D94AE80868B7D873EC0BF042E900EBD3
:1002B000E9FF01EBEAFFEF5005E1300E006E000EA2
:1002C000016E08D0A8D8300EE66E000EE66E0CEC7B
:1002D0000BF044E9020EE66EE66AFD0EE66E1E0EB7
:1002E000E66EE9D805E097D8C2EC03F042E929D0E0
:1002F0000A6A160EF36EF46AF3500A5C000EF454A8
:100300001BE2A6D851EC0BF042E9BDC0C5F0BEC05F
:10031000C6F0BFC0C7F00001C5510B6EC6510C6ED0
:100320000BEBE6FF0CEBE6FF93D8C5D803E18AEBB5
:1003300008F002D00A2ADDD76ED808EBE6FFE3DE2C
:1003400043E9096E09EBE6FF54DF41E94BE9E7CFEA
:10035000D9FF12000001029102976EDEEDEF05F069
:10036000A1D859D885D82DEC0BF044E981D802D812
:1003700042E98ED097D8FB0EE66E1E0EA2D8000181
:1003800000A704D0F90EE66E1E0E9BD844D860EC90
:100390000AF042E97DD044D870D86AD8020EE66EE1
:1003A000D950010FE66EDACFE6FF6EEC0DF045E9AD
:1003B0005FD872D035D861D8C60EE66E1C0EE66ED8
:1003C00057D82DEC0BF044E9120E025C08E1E00E68
:1003D0000114600804E1EC0EE66E1E0E15D0120E3C
:1003E000025C04E1E00E0114400807E0240E025C08
:1003F00008E1E00E0114200804E1DF0EE66E1E0E97
:1004000003D0CC0EE66E1E0EE66E32D8DFEC0AF09C
:1004100044E92ED841D000EBE6FF01EBE6FF1200E5
:10042000D9CFE6FFE1CFD9FF1200D950030FE66E16
:10043000DACFE6FF040E00010024C56F000E012094
:10044000C66FC5C0E6FFE66E2AEC0DF044E9120067
:10045000F76A0A34FE0BF66EF7364B0EF6261D0EC3
:10046000F7220900F5CFE6FF0900F5CFE6FF1200FD
:10047000070EE66E000EE66E120081E942E8D950E2
:10048000010FE66EDACFE6FF9EEC0DF042E91200B6
:1004900041E9E7CFD9FF12006DDF42E943E9E7CF39
:1004A000D9FF1200BDDF83E91200B5DF43EC0BF08A
:1004B00042E9F3501200AFDFA2EC0AF046E900096E
:0E04C0001200E66EA8DFDFEC0AF044E912003D
:0204CE00EB0E33
:1004D000D76EDB0ED66EF2941200F2A4FED7120095
:1004E000C7D982E90F0E00140A0A13E0040A11E0CA
:1004F000070A0DE0020A0BE0060A09E0020A07E01B
:10050000090A07E0030A05E0020A05E102D0010E2C
:1005100003D0000E01D0000E41E9E7CFD9FF120051
:10052000A7D9C1D99AEC06F0016E015021E0A5D9F6
:10053000150EE66E4C0EE66E030ED9D9030E0001C1
:100540009E5D3BE1550E9F5D38E1A051026EA151C9
:10055000036E93D9C60EE66E53EC10F041E900012C
:10056000010E9E6FA11D9F6FCCD9016E015003E15A
:100570000001028322D0150EE66E0D0EE66E010E0E
:10058000B3D99E051AE1CC0E9F5D17E176D9080E0E
:10059000035C03E0940E035C04E100010281029716
:1005A0000CD08F0E035C09E102EBE6FF99DF41E915
:1005B000000903E000010281028744E9E7CFD9FF87
:1005C000120056D970D9E0EC06F0016E015003E13B
:1005D0000001028339D0020EE66EE66AE00EE66E96
:1005E000200E7DD96CD93FD9A4EC0BF042E989D912
:1005F000320EE66E4C0EE66E080E79D9050E00013D
:100600009E5D22E39F5102E1030E0BD0C00E9F15A9
:1006100002E1020E06D03F0E9F1502E0040E01D04B
:10062000050E026E025039D9EF50C1080DE10228C3
:1006300034D9EF50036E03EBE6FF52DF41E90009C6
:1006400003E000010281028744E9E7CFD9FF1200ED
:100650000FD982E9E80EE66E200EE66E73EC0AF022
:1006600042E9005002E15CDF06D0000403E058DFFD
:10067000000102A1A6DF000102A111D028DF0001C4
:10068000AA690001066B020E005C07E1F40EE66E3B
:10069000200EE66EB0EC01F042E9000E05D002A398
:1006A00002D0080E01D0070E41E9E7CFD9FF1200B2
:1006B000DFD881E941E8000102A709D0020EE66E09
:1006C000E66AE60EE66E200E0AD9F9D80BD0040EC3
:1006D000E66EE66AE20EE66E200E01D9C4D888EC1A
:1006E0000BF042E9F5D8016E015008E0150EE66EF8
:1006F0000D0EE66E0B0EF8D89E5102E10001062B9E
:10070000E6DE42E9E7CFD9FF1200F6D80C0EFED89C
:1007100045EF04F0ADD881E941E8016A0C0EF36EB3
:10072000F46AF350015C000EF45405E20150B5D8B0
:10073000EF6A012AF3D742E9E7CFD9FF120000019F
:1007400002A117D00651050802E202911200FF0E25
:100750000001AA5D04E1CE6ACF6A9E9008D09EA0F7
:1007600002D0AA2B9E901D0EAA5D01E21200AA6B78
:100770009FDF1200CE6ACF6A9E900001AA6B000133
:10078000066B120075D883E944E8056A00EBE6FFC2
:1007900001EBE6FFFDEC0CF042E9000902E1010E7D
:1007A0005ED0000102B10AD0020EE66E51DF41E9CF
:1007B000036E000102B102D0035051D054D800EBB7
:1007C000E6FF01EBE6FF2AEC0DF044E9000102B779
:1007D00005D049D888EC0BF042E901D070D878D820
:1007E000036E035002E10C0E3AD0046A640E045CFE
:1007F0002FE2150EE66E01C0E6FF0B0E75D89E5176
:1008000027E0050E9E5D02E2040E29D0000100B52E
:1008100014D029D8CFEC0BF042E900019E5102E13F
:10082000050E1DD0000102B704D01DD8B8EC0BF0A6
:1008300003D019D823EC0CF042E95ED89EC0E6FF45
:100840009F0EE66E000EE66E20D8042A052ACED74B
:10085000055002E1060E03D08DDF39DE090E45E9B1
:10086000E7CFD9FF12009E0EE66E000EE66E120074
:10087000D9CFE6FFE1CFD9FF1200F20EE66E200ECF
:10088000E66E73EC0AF042E912006EEC0DF045E9F9
:1008900033D8BAEC01F042E91200EA6A9E0FE96E21
:1008A000000EEA22120081E943E80001029102975A
:1008B000029312004AEC06F045E900011200E66AD4
:1008C000030EE66E000E22D8E4EC0BF045E91200B0
:1008D000CADFA4EC0BF042E900DE81EF04F016D889
:1008E000BFEC0AF046E9120011D85AEF04F00ED816
:1008F0004AEC06F045E91200070EE66E000EE66EC1
:100900001200B1DF12EC06F042E91200E66E33EF9E
:0209100004F0F1
:0E091200040120511F0B010801E012002051CA
:10092000600BE842E842E842E842E842010801E0A0
:100930001200245103E0240501E012002151230A92
:1009400039E0010A33E0030A25E0010A1CE0240A29
:1009500031E0070A2FE0010A2DE0030A0EE0010A48
:1009600001E0120031D90001960EB76F000EB86F8A
:100970000001C2930001080E17D026D90001960E7F
:10098000B96F000E05D020D900018B0EB96F000E93
:10099000BA6F120019D900018B0EB76F000EB86F35
:1009A0000001C2930001070EBB6F12000DD922C4D3
:1009B00092F01200120000018B6BC20E8C6F010EC0
:1009C0008D6F8E6B8F6B906B080E916F846B836B4A
:1009D0001A0E726E1E0E736E0401000E166F050E57
:1009E000176F400E146F0401196F080E1A6F050E71
:1009F0001B6F880E186F0401480E1E6F050E1F6FC7
:100A0000400E1C6F1200E4D884E90001836B0401DE
:100A100018BF24D00050195D02E21951006E000188
:100A2000836B0050835D13E28351EA6A080FE96E1D
:100A3000050EEA22EF50E66E83510124E96E000EA6
:100A40000220EA6EE552E750EF6E832BEAD70401ED
:100A5000400E196F1817187D880E18130001835166
:100A600041E9E7CFD9FF12009ED812E1036AA1D86D
:100A700002E1F45009E000EBE9FF01EBEAFF002A94
:100A8000000E0122EF50F3E176D88A6B010E846FDD
:100A900097D089D813E1036A8CD802E1F4500AE0B8
:100AA00000EBF6FF01EBF7FF002A000E0122080021
:100AB000F550F2E160D8010E8A6F846F81D088D83A
:100AC00081E941E804011CBF55D0030E0001845D9B
:100AD00001E1846B84514EE0020E845D03E1040168
:100AE0001D6B3FD0840540E189510001C56FC66B85
:100AF000C5514008000EC65502E2400E02D000016A
:100B00008951016E01EB1DF401500001895D896F6F
:100B1000480E876F050E886F8A050AE1015011E0C3
:100B200085C0F6FF86C0F7FF0800F55030D8F6D72D
:100B3000015007E085C0E9FF86C0EAFFEF5027D8E3
:100B4000F7D70001895110E104011D510001C56F63
:100B5000C66B400EC51905E1C65103E10001020E46
:100B600002D00001030E846F400E04011C171C7D8F
:100B7000880E1C1325D00350005E000E015A00EBB6
:100B800085F001EB86F003040001896F120087C035
:100B9000E9FF88C0EAFFEF6E872B000E8823852BC4
:100BA00086230106120014D883E941E8000184512C
:100BB0001200032AFF0EF36EF46AF35003181200BA
:100BC00042E9E7CFD9FF12000001030EB66F120011
:0A0BD000D9CFE6FFE1CFD9FF1200F4
:060BDA00080EB86E0001D8
:100BE00000B9B888400EE66E020EE66E3C0EE66E68
:100BF00007EC10F043E912003AD982E9FE0ED76EF5
:100C0000880ED66EF2949EBA03D0F2A4FCD703D01D
:100C10000050AE5C02E0000E01D0010E41E9E7CFCA
:100C2000D9FF120024D983E944E880EB04F081EB7A
:100C300005F0010E066E8A8400EBE9FF01EBEAFF86
:100C4000EF04036E033420E2ACA2FED7042A000EA8
:100C5000052204EBE9FF05EBEAFFEF50AD6E04EB74
:100C6000E9FF05EBEAFFEFCFE6FFC6DF41E9000948
:100C700002E1066A09D0033405E20350000802E2EB
:100C80002A0EFAD80306DED78A94065045E9E7CF44
:100C9000D9FF1200ECD886E945E8066A83EB09F033
:100CA00084EB0AF0F2940150AE0802E2AE0E016E3F
:100CB00001500001C2D8C6C0C5F0C66BC5C0D7FF81
:100CC0000150BBD8C551D66E9FD8C6C0C5F0C66B03
:100CD000C551076E99D8C551086E03EBE9FF04EBC7
:100CE000EAFFEF6A066A0250065C19E29EBA03D078
:100CF000F2A4FCD714D0ABB412D0ABB210D0092AF6
:100D0000000E0A2209EBE9FF0AEBEAFFAECFEFFF84
:100D10008A8207EBD7FF08EBD6FF062AE4D703EB5E
:100D2000E9FF04EBEAFF06EBEFFF8A9246E9E7CF23
:100D3000D9FF120095D802E08B8C01D08B9CA1D8F2
:100D400002E08B9C01D08B8CA0D802E08B9C01D060
:100D50008B8C9BD802E08B8C01D08B9C92D802E0CC
:100D60008B8C01D08B9C8DD802E08B9C01D08B8C1E
:100D70008CD802E08B9C01D08B8C87D802E08B8CC6
:100D800001D08B9C7ED802E08B8C01D08B9C79D8D3
:100D900002E08B9C01D08B8C8A968A9A780EE66E44
:100DA00038EC10F041E9AB8EAC8A8A9482AE000C2C
:100DB000000100AB04D0E6681FDF41E91200010C1E
:100DC0004FD802E08B8C01D08B9C8A868A8A960E43
:100DD00053D88B7C8A968A9A960E4ED8AB8EAC8A64
:100DE0008A9482AE000C000100AB04D0E66804DFF8
:100DF00041E91200010C780EE66E38EC10F041E982
:100E000000010051100B1200040EE66EE66A770E28
:100E1000E66E010EE66E0050E66EE66A8DEC0CF0B2
:100E200051EC0CF0E552E5CFC6F0E7CFC5F000017C
:100E3000FF0ED880C557C6571200C56FC66B770E18
:100E4000C603F3CFC6F0C551C627770EC503F3CF4F
:100E5000C5F0F450C627FF0ED880C557C6571200FC
:100E60008A84AB9EAC9A00010051100B1200D9CFBE
:100E7000E6FFE1CFD9FF1200E66E53EC10F041E936
:100E800012008A868A8AFBEF06F08A968A9AFBEF1E
:020E900006F06A
:0E0E920004012051600BE842E842E842E842C9
:100EA000E842000901E012002151070A3FE00B0A65
:100EB0003DE0070A32E0010A23E00B0A1FE0020AC4
:100EC0001DE0030A19E0080A10E0010A0CE00F0A0D
:100ED00008E0030A01E0120015D90001040EC16FF9
:100EE000120097EF07F0CEEF07F00CD90001C30E08
:100EF000B76F000EB86F0BD0EFEF07F021EF08F0DF
:100F000005D90001B86BC40FB76F000EB8230001FC
:100F1000C2930001010EBB6F1200F8D8EA6AC40F39
:100F2000E96E000EEA2222C4EFFF12001200800ECA
:100F30000401205D32E12351030A1FE0010A0AE0A7
:100F4000030A29E1DFD80001770EB76F1D0EB86FD5
:100F5000120E1ED0C1D8180EF6261E0EC6D8020ECE
:100F60000001F76AB725F66EB851F7220900F5CFF0
:100F7000BBF00A00F5CFBCF00ED0AED81C0EF626A2
:100F80001E0EB3D8B7C0F6FFB8C0F7FF0800F55083
:100F90000001BB6FBC6B0001C2831200B3D80F0EFF
:100FA000E66E710EE66E0F0EE66E51EC0EF043E942
:100FB000010EE66EC40EE66E000EE66E51EC0EF00B
:100FC00043E922C4C3F00401225104E10001050EEB
:100FD000C16F12000001060EC16FDBEF04F00401C7
:100FE000286B296B040120511F0B020A0FE0030A32
:100FF0000BE0010A18E186D8040128810001C2A192
:1010000012D0040128830FD07DD80DD04BD801E039
:10101000010E56D8B9C0E9FFEA6EEF50040B03E0A9
:101020000401010E286F0001B6050AE10001280E37
:10103000B76F040EB86F0001C2930001020EBB6FC0
:101040001200040122050EE120511F0B00090AE1E4
:1010500059D8030E0401215D03E10001C28102D0D1
:101060000001C291040122511CE120511F0B020812
:1010700018E124510F0B000914E014D801E0010E0F
:101080001FD8030E0401215D04E1840E36D8EF6EF3
:10109000120024AF03D031D8EF6A1200880E2DD889
:1010A000EF6E120033D80F0B080DF3500001C66B22
:1010B000000FC56F040EC62304012451800B1200DB
:1010C000040DF3500001C5250001B96F000E0001A9
:1010D000C6210001BA6F120015D804012251F66E24
:1010E000F76AD890F636F7361200F7220900F5CFE6
:1010F000B7F00A00F5CFB8F01200B9C0E9FFBAC0E6
:10110000EAFF12000001010EB66F1200FBDF0401BE
:041110002451120054
:0C1114006C500BE1040100513C0BE84260
:10112000E8420D0802E19CEF08F0CCEF08F0040E55
:101130006C5C01E140D8120010D941E80001B56BA8
:10114000B66BBB6BBC6B49EC07F0016A010EF36E2A
:10115000F46AF350015C000EF45419E20001B65138
:1011600016E1F76A0134FE0BF66EF736240EF6260A
:101170001E0EF7220900F5CFC5F00800F5CFC6F026
:10118000C6C0FAFF0001C5511400012ADFD794D868
:1011900042E9E7CFD9FF1200020E0001B55D09E177
:1011A00061D8040100BD02D0C80E01D0880E006FC6
:1011B000120095EF09F0040E0001C15D09E122C49F
:1011C0006EFF6E50000802E2050E01D0030EC16FE3
:1011D0000001B50509E10AD8040104BD02D0C80E1A
:1011E00001D0880E046F120095EF09F0B6D842E8DE
:1011F0000001080EBB5D000EBC5905E2BB51016E3B
:10120000BC51026E03D0080E016E026A0401049301
:1012100004910250041301EB05F401500001BB5F7F
:101220000250BC5B280EB96F040EBA6F0001C2A356
:101230000BD00150021012E0B7C0F6FFB8C0F7FFA4
:101240000800F5507AD8F5D70150021007E0B7C072
:10125000E9FFB8C0EAFFEF5070D8F6D743E9E7CF0F
:10126000D9FF12007AD842E8030E04010015026E7D
:101270000151016EBB0EE96E000EEA6E0001EE50E8
:101280000124BB6FED500220BC6F280EB76F040E17
:10129000B86F015002100CE0B7C0E9FFB8C0EAFF18
:1012A000EF50B9C0E9FFBAC0EAFFEF6E5CD8F1D7E2
:1012B00043E9E7CFD9FF12006D980001B65105E16F
:1012C00044D8840E006F04011DD0040120AF1CD04F
:1012D0000001BB510401265D0001BC5104012759E6
:1012E00004E226C4BBF027C4BCF080DF0001010E7D
:1012F000B56F2BD8800E006F0401280E066F040E08
:10130000076FC80E046F12000001020EB56F0401D2
:10131000056BC80E046F0401080E016F280E026FE2
:10132000040E036FC80E006F12000001B56B0DD8DC
:10133000880E006F0401046B1200B9C0E9FFBAC047
:10134000EAFFEF6E0001B3EF09F00401080E016F30
:10135000200E026F040E036F1200D9CFE6FFE1CF1B
:10136000D9FF81E91200B92B000EBA23B72BB8239D
:061370000106025A120002
:0A1376000001CA51CB1104E1100E72
:10138000CA6F270ECB6FCA07000ECB5B6DA205D0CC
:10139000CA51CB1116E18A7012000001C151060A30
:1013A0000FE0030A0BE0060A09E0010A0AE0030A5B
:1013B00005E0010A01E012008A9012008A80120002
:1013C0008A801200D9CFE6FFE1CFD9FF81E945E855
:1013D000D2DF060E0001C15D64E36D50020B61E1D6
:1013E000ACD843EC0BF042E9F350016EF450026EBE
:1013F0005A0E0124036E000E0220046E00010150FB
:101400002908C56F000E0254C66FC5C0E6FF03EB86
:10141000E6FF04EBE6FF03EC05F043E9000941E0D9
:1014200000018351056E05500126000E0222290E8F
:10143000015C000E025833E25A0E0124E96E000EE0
:101440000220EA6EEF6A000100A306D003EBE6FF7C
:1014500004EBE6FF35D842E90D0EE66E6ED8F8ECE7
:101460000AF043E9F350036EF450046E0350041085
:1014700018E000010051020B09E00051080B06E0E2
:101480006D0EE66E1F0EE66E2ED842E903EBE9FF05
:1014900004EBEAFFEF6A51D850EC01F042E9000199
:1014A0005A6B46E9E7CFD9FF120000015A6B1200D0
:1014B000B1EC0DF06FBE02D0CDEC0DF05FEF05F09A
:1014C00033D80001845103E021D8FBE208D000EBBF
:1014D000E6FF01EBE6FF34EC05F042E9E9DF43E922
:1014E000E7CFD9FF120020D80001845103E00ED8C5
:1014F000FBE208D000EBE6FF01EBE6FF49EC05F06C
:1015000042E9D6DF43E9E7CFD9FF1200D1DF032A52
:10151000000E042203EBC5F004EBC6F00001C55138
:10152000E808030EC6551200D9CFE6FFE1CFD9FF78
:1015300083E942E8036A046A12005A0EE66E000E5E
:04154000E66E120041
:0C154400FC0EE3CFF6FFFD0EE3CFF7FF37
:10155000FE0EE3CFE9FFFF0EE3CFEAFFFA0EE35002
:1015600003E1FB0EE35009E0FA0EE30602E2FB0E94
:10157000E3060900F550EE5CF1E0F36E1200FC0E9C
:10158000E3CFF6FFFD0EE3CFF7FFFE0EE3CFE9FF5B
:10159000FF0EE3CFEAFFE9CFF3FFEACFF4FFFA0E45
:1015A000E35003E1FB0EE35009E0FA0EE30602E22A
:1015B000FB0EE3060900F5CFEEFFF1D71200FC0E9B
:1015C000E3CFF6FFFD0EE3CFF7FFFE0EE3CFE9FF1B
:1015D000FF0EE3CFEAFFE9CFF3FFEACFF4FFEE66B9
:1015E000FED7ED520900F5CFEFFFEE66FBD71200F4
:1015F000FE0EE3CFE9FFFF0EE3CFEAFFFD0EE3505F
:10160000EF5C05E0EE66FAD7F36AF46A04D0E9CF3E
:10161000F3FFEACFF4FF1200D9CFE6FFDACFE6FFFF
:10162000FA0EE3CFD9FFFB0EE3CFDAFFFC0EE3CFD8
:10163000E9FFFD0EE3CFEAFFE9CFF3FFEACFF4FFC6
:10164000DECFEFFFEE66FCD7FF0EE3CFDAFFE55209
:10165000FF0EE3CFD9FFE5521200FC0EE3CFF6FFF9
:10166000FD0EE3CFF7FFFE0EE3CFE9FFFF0EE3CF62
:10167000EAFFE9CFF3FFEACFF4FF0900F5CFEFFF70
:10168000EE66FBD71200FE0EE3CFE9FFFF0EE3CFBD
:10169000EAFFF36AF46AEE5203E0F34AF42AFBD756
:1016A0001200FF0EE3CFF7FFE552FF0EE3CFF6FF88
:1016B000E552E56AE66AE66AE66A0900F55209E07B
:1016C000FD0EE32A05E1FE0EE32A02E1FF0EE32A06
:1016D000F4D7FD0EE3CFBDF0FE0EE3CFBEF0FF0E5C
:1016E000E3CFBFF01200FE0EE3CFE9FFFF0EE3CF22
:1016F000EAFFE9CFF3FFEACFF4FF610EEF5C05E606
:101700007B0EEF5C02E7DF0EEF16EE52F6E1120001
:10171000FE0EE3CFE9FFFF0EE3CFEAFFEFCFF3FFCB
:10172000030EEF26F36EE926000EEA22040EEDCF3B
:10173000EBFFF32EFCD7680EEC6E6A0EEC6EF10E2A
:10174000EC6EFD0EEB501200FE0EE3CFE9FFFF0E34
:10175000E3CFEAFFEFCFF3FFF3CFF4FFF42AF4CFA8
:10176000EEFFE86AEE24F32EFDD7EF6EF450120080
:10177000FE0EE3CFE9FFFF0EE3CFEAFFEFCFF3FF6B
:10178000030EF35E0AE009E6F3CFF4FFF3CFEEFFBA
:10179000030EEBCFEEFFF32EFCD7F4501200FE0E3B
:1017A000E3CFE9FFFF0EE3CFEAFFEFCFF3FFF3064E
:1017B000F3CFF4FFF3CFEEFFE86AEE24F32EFDD76C
:1017C000EF18D8B4F4501200D9CFE6FFDACFE6FF15
:1017D000FC0EE3CFE9FFFD0EE3CFEAFFF90EE3CF06
:1017E000F4FFEFCFF3FFEF50E926000EEA22030EDD
:1017F000F4B0E82AD96EE82AEDCFEBFFF32EFCD740
:10180000EFCFF3FFD950EF26FA0EE3CFD9FFFB0E4F
:10181000E3CFDAFFE86AF4A0F350DE10EC6EDECF1F
:10182000ECFFDECFECFFF4B0F3CFECFFE552E7CFF7
:10183000DAFFE552E7CFD9FFF4B002D0FD0E01D0B8
:10184000FC0EEB501200D9CFE6FFFD0EE3CFE9FF0F
:10185000FE0EE3CFEAFFEFCFF3FF010EEB503F0B9D
:10186000030ED8B4E82AD96EF35E0AE009E6F3CF96
:10187000F4FFF3CFEEFFD950EBCFEEFFF32EFCD702
:0A188000E552E7CFD9FFF450120043
:06188A0043E8D9CFE6FFA0
:10189000DACFE6FFE1CFD9FFE2CFDAFF89E9066AC6
:1018A0001200F3DF068001D0F0DF01AE5EEF0CF036
:1018B000006C011EE86A012206B0067E03AE66EFE8
:1018C0000CF0026C031EE86A0322067ED2EC0CF0D8
:1018D00003BE88EF0CF006AE08D0026C031EE86A67
:1018E0000322046C051EE86A052206B006D084EBCC
:1018F00000F085EB01F006A004D082EB00F083EB52
:1019000001F0E552E5CFDAFFE7CFD9FF45E9000C5A
:1019100006BE6DEF0CF0E9DFFF0C44E8D9CFE6FF1F
:10192000DACFE6FFE1CFD9FFE2CFDAFF8AE980EB39
:1019300004F081EB05F082EB06F002500402F45053
:10194000016EF350006E0350076E0502F450036EF3
:10195000F350026E07500402F3500126F4500222A5
:10196000E86A032206500502F3500126F4500222D1
:10197000E86A0322E552E5CFDAFFE7CFD9FF46E96F
:10198000000C43E8D9CFE6FFDACFE6FFE1CFD9FF7D
:10199000E2CFDAFF89E9066A1200F3DF068003D09E
:1019A000F0DF01D00682056A046A100EE76ED89057
:1019B00002360336043605360050045C01500558E3
:1019C00005E30050045E0150055A022AE72EF0D7C5
:1019D00006B2120006B006D084EB00F085EB01F0F1
:1019E00006A004D082EB00F083EB01F0E552E5CFD6
:0A19F000DAFFE7CFD9FF45E9120046
:0619FA00FE0EE3CFE9FF41
:101A0000FF0EE3CFEAFFF36AEE5006E018D8FCE0E1
:101A100009D806E1F32AF8D7F3B002D0F350120048
:101A2000E86A1200F452C60F0A0F06E2F450B90F2A
:101A3000060F02E2D8941200F450D8841200F46E1B
:101A4000200806E0F450090803E0F450D89412008E
:101A5000D8841200D9CFE6FFDACFE6FFFC0EE3CF41
:101A6000E9FFFD0EE3CFEAFFFC0EE3CFD9FFFD0E49
:101A7000E3CFDAFFF36ADE5007E0E1DFFCE0D2DF1C
:101A80001FE1F32AEE6EF7D7EF6AF3B019D0F342F5
:101A9000FC0EE3CFE9FFFD0EE3CFEAFFFA0EE3CF42
:101AA000D9FFFB0EE3CFDAFFF3CFDEFFEF5206E004
:101AB0000FD8E83ADF6E0CD8DE12F8D7F35001D019
:101AC000E86AE552E7CFDAFFE552E7CFD9FF120027
:101AD000EE50C00FD8A0070F090F1200D9CFE6FFB4
:101AE000DACFE6FFFC0EE3CFE9FFFD0EE3CFEAFF1E
:101AF000FB0EE3CFF3FFF90EE3CFD9FFFA0EE3CFEE
:101B0000DAFFF3520FE0EF50F00BE83A12D8DE6E36
:101B1000EE500F0B0ED8DE6E200EDE6EF32EF3D7D6
:101B2000DD52DF6AE552E7CFDAFFE552E7CFD9FFB2
:101B30001200360FD8B2070FFA0F1200FE0EE3CFD5
:101B4000E9FFFF0EE3CFEAFF3F0EF86EFF0EF76EE0
:101B5000FE0EF66E0900F5CFEEFF0900F5CFEEFFA1
:021B6000120071
:0E1B62006DA60CD80001C10508E16DBA06D0D1
:101B7000686A696A69806988020EC16F12006D6ABD
:101B8000696A6D860001010EC16F12006D6A696A93
:101B90000001C16B1200C6EF0DF00001C15101E15F
:101BA00012006850040B04E06950040B01E038D8BF
:101BB0006DB212006850010B04E06950010B01E0A6
:101BC00050D86850100B04E06950100B01E024D885
:101BD0006850400B04E06950400B01E037D8685072
:101BE000200B04E06950200B01E032D86850020B52
:101BF00004E06950020B01E032D8030E0001C15D20
:101C000001E212006850080B06E06950080B03E07F
:101C10008AEC08F068961200698468986D82120058
:101C20006D926994689412000001C2A10ED0F8DF91
:101C30006D840001080EC86F070EC96FC807000E3B
:101C4000C95BC851C911FAE16D941200689C120079
:101C500070A003D095EC09F07090689A1200689219
:101C600012006A6A686A9F0E6B6E7B0E696E6E6AFE
:101C70000F0EE66E710EE66E0F0EE66E12D843E999
:101C8000160E706E68A602D06896FCD76D9895EC1B
:101C900009F00001C2910001C36B0001030EC16F86
:101CA0001200D9CFE6FFE1CFD9FF84E901EBE9FFCC
:101CB00002EBEAFF005003E0EE6A0006FBD741E9C1
:061CC000E7CFD9FF12007E
:0A1CC6004F4244444941472E4E4569
:101CD000542076312E323720627920416C6578208D
:101CE0005369646F72656E6B6F003F004F4B004528
:101CF0004C4D3332332076322E3020636F6D70615D
:101D00007469626C650044415441204552524F52FF
:101D1000003C44415441204552524F52004E4F2006
:101D200044415441004552524F52004642204552D0
:101D3000524F520042555320425553590050726F32
:101D40006772616D204572726F7200681F631F5F5A
:101D50001F5A1F551F501F4B1F461F411F3D1F3845
:101D60001F331F2E1F291F241F1F1F1A1F151F106F
:071D70001F0C1F071F021FDB
:091D77001201000202000008D86C
:101D8000040A0000000102030109024300020100ED
:101D90008032090400000102020100052400100144
:101DA00004240202052406000105240100010705A0
:101DB000820308000209040100020A00000007056E
:101DC00003024000000705830240000004030904E9
:101DD00018034F006200640044006900610067005E
:101DE0002E004E00650074001A034F0042004400AC
:101DF0003200200041006400610070007400650042
:101E00007200160331003700340031003500310014
:101E10003200340035003500891D891DCC1DD01DD0
:061E2000E81D021E12097C
:0A1E26000F0EC1128A6AF19E080E29
:101E3000936E8150080B02E0000E01D0010E0001EC
:101E40000099E8B00089800E946EF29EF29C850E97
:101E5000D56EF28AB50ECD6E9D801200D9CFE6FF09
:101E6000E1CFD9FF81E942E8D950010FE66EDACF20
:101E7000E6FF9EEC0DF042E9120E025C0AE11F0E35
:101E800001140001C56F040EC55D03E20001008B63
:101E900002D00001009B43E9E7CFD9FF1200140EE6
:101EA0006F6E0001C16B0001C26B0001C36BBBDF31
:101EB00055EC0AF0AAEC01F02EEF0FF0F0DF58EC31
:0C1EC0000AF0E2EC09F09FEC03F0F9D707
:041ECC002C20756EE3
:101ED000737570706F727465642063686970002C2C
:101EE0002050494331384632353530002C20504996
:101EF0004331384632343535000A000D0041540074
:101F00003E004154403200415440310041545A0097
:101F100041545357004154535400415453520041CB
:101F200054534900415453480041545044004154D3
:101F30004D410041544C310041544C300041544912
:101F40000041544831004154483000415446490052
:101F5000415446440041544531004154453000410C
:0F1F6000544400415442440041544152000A008D
:101F70002A0EF66E000EF76E000EF86E00010900D4
:101F8000F550B06F0900F550B16F03E1B06701D0B3
:101F90003DD00900F550AB6F0900F550AC6F09005A
:101FA000F550AD6F09000900F550E96E0900F550D4
:101FB000EA6E090009000900F550AE6F0900F550FE
:101FC000AF6F09000900F6CFB2F0F7CFB3F0F8CF4A
:101FD000B4F0ABC0F6FFACC0F7FFADC0F8FF000136
:101FE000AE5302E1AF5307E00900F550EE6EAE07C5
:101FF000F8E2AF07F9D7B2C0F6FFB3C0F7FFB4C03D
:0E200000F8FF0001B007000EB15BBFD7120061
:02200E00D9CF28
:10201000E6FFE1CFD9FF84E9AC6AAB6A02A005D044
:10202000AC8802A404D0AC8E02D002B8AC8402A268
:1020300002D0AC8CAB8C02A602D0AB8801D0AB8AAC
:1020400002AC02D09D8A01D09D9A02AE02D09D883A
:1020500001D09D9800EBAFFF000101EBC5F0C66B0E
:10206000C5C0B0FFAC8AAB8E41E9E7CFD9FF120003
:10207000FF0EE3500001CD6FEE0E02D0F20E000015
:10208000E76EE72E41EF10F00C0E0001CC6FE76A0F
:10209000E72E48EF10F0CC2F47EF10F00001CD2FC6
:0620A0003EEF10F01200FB
:0A20A600FF0EE3500001CD6F480E5D
:1020B00001D04C0EE76EE72EFED7E76AE72EFED77B
:0620C000CD2FF7D712003E
:0A20C60013EE00F023EE00F0F86ABC
:1020D000B8EC0FF083EC10F05EEC0FF0FBD71200C1
:1020E000018102010000013E425553494E49543AD4
:0720F00020002E004F4B0001
:0820F80000EE00F00F0EEE6A8D
:06210000EA62FDD71200A7
:022106001200C5
:022108000000D5
:020000040030CA
:0100000034CB
:010001000EF0
:010002003FBE
:010003001EDE
:0100040000FB
:01000500807A
:01000600C138
:0100070000F8
:0100080008EF
:0100090000F6
:01000A000FE6
:01000B00E014
:01000C000FE4
:01000D0040B2
:00000001FF
